:020000040800F2
:1000000000060020A1020008FD0F00087D0F000877
:10001000D50F00087D0F0008A90F0008A3020008F3
:10002000A3020008A3020008A3020008DD290008BB
:10003000A3020008A3020008A3020008A30200080C
:10004000A3020008A3020008A3020008A3020008FC
:10005000A3020008A3020008653E0008913E0008C4
:10006000BD3E0008E93E0008153F0008A302000855
:10007000A3020008A3020008A3020008A3020008CC
:10008000A3020008A3020008A3020008A3020008BC
:10009000A3020008A3020008A3020008413F0008D1
:1000A000A3020008A3020008A3020008A30200089C
:1000B000A3020008A3020008A3020008A30200088C
:1000C000A3020008A3020008A3020008A30200087C
:1000D000A3020008A3020008194000082D400008F0
:1000E000A53F0008A3020008A3020008A30200081D
:1000F000A3020008A3020008A3020008A30200084C
:10010000A3020008A302000855400008A30200084B
:10011000A3020008A3020008A3020008A30200082B
:10012000A3020008A3020008A3020008A30200081B
:10013000A3020008A3020008A3020008A30200080B
:10014000A3020008A3020008A3020008A3020008FB
:10015000A3020008A3020008A3020008A3020008EB
:10016000A3020008A3020008A3020008A3020008DB
:10017000A302000849350008A3020008A3020008F2
:10018000A3020008A302000841400008A3020008DF
:10019000A3020008A3020008A3020008A3020008AB
:1001A000A3020008A3020008A3020008A30200089B
:1001B000A3020008A3020008A3020008A30200088B
:1001C000A3020008A3020008A3020008A30200087B
:1001D000A302000835350008A3020008A3020008A6
:1001E000A3020008A3020008A3020008A30200085B
:1001F000A3020008A3020008A3020008A30200084B
:10020000A3020008A3020008A3020008A30200083A
:10021000A3020008A3020008A3020008A30200082A
:10022000A3020008A3020008A3020008A30200081A
:10023000A3020008A3020008A3020008A30200080A
:10024000A3020008A3020008A3020008A3020008FA
:10025000A3020008A3020008A3020008A3020008EA
:10026000A3020008A3020008A3020008A3020008DA
:10027000A3020008A3020008A3020008A3020008CA
:10028000A3020008A3020008A3020008A3020008BA
:10029000A3020008A3020008A3020008A3020008AA
:1002A00002E000F000F8FEE772B63A4880F30888F2
:1002B000394880F3098839484EF60851CEF20001DA
:1002C000086040F20000CCF200004EF63471CEF22D
:1002D00000010860BFF34F8FBFF36F8F40F2000043
:1002E000C0F2F0004EF68851CEF200010860BFF374
:1002F0004F8FBFF36F8F4FF00000E1EE100A4EF604
:100300003C71CEF200010860062080F31488BFF330
:100310006F8F02F021FC02F0C3FB03F05DFB4FF096
:1003200055301F491B4A91423CBF41F8040BFAE784
:100330001C49194A91423CBF41F8040BFAE71A499B
:100340001A4A1B4B9A423EBF51F8040B42F8040B69
:10035000F8E700201749184A91423CBF41F8040BC6
:10036000FAE702F0DBFB03F0BBFB144C144DAC428C
:1003700003DA54F8041B8847F9E700F041F8114C00
:10038000114DAC4203DA54F8041B8847F9E702F038
:10039000C3BB00000006002000220020000000086F
:1003A00000000020000600209044000800220020E9
:1003B0005C22002060220020D44F0020A002000810
:1003C000A0020008A0020008A00200082DE9F04FDA
:1003D0002DED108AC1F80CD0D0F80CD0BDEC108AED
:1003E000BDE8F08F002383F311882846A047002042
:1003F00001F0DAFEFEE701F055FE00DFFEE7000047
:1004000038B500F0D7FC30B1164B00220E211A721D
:100410005A729972DA7202F0A1FA054602F0D4FA21
:100420000446D0B9104B9D4219D001339D4241F290
:10043000883512BF044600250124002002F098FAF6
:100440000CB100F059F800F039FD00F0F9FB284636
:1004500000F004F900F050F8F9E70025EDE7054653
:10046000EBE700BF00220020010007B008B500F054
:10047000B3FBA0F120035842584108BD07B541F233
:100480001203022101A8ADF8043000F0C3FB03B051
:100490005DF804FB202310B583F311881248C3686C
:1004A0000BB101F007FF0023104A4FF47A710E4898
:1004B00001F0C4FE002383F311880D4C236813B1AF
:1004C0002368013B2360636813B16368013B636089
:1004D000084B1B7833B9636823B9022000F070FC25
:1004E0003223636010BD00BF602200209504000825
:1004F0007C23002074220020F8B5514B514A1C4641
:100500001968013100F09B8004339342F8D162688E
:100510004D4B9A4240F293804C4B9B6803F1006331
:1005200003F500339A4280F08A80002000F0A2FB9D
:100530000220474B187000F041FC464B0021D3F8D5
:10054000E820C3F8E810D3F81021C3F81011D3F84D
:100550001021D3F8EC20C3F8EC10D3F81421C3F821
:100560001411D3F81421D3F8F020C3F8F010D3F805
:100570001821C3F81811D3F81821D3F8802042F0BD
:100580000062C3F88020D3F8802022F00062C3F814
:100590008020D3F88020D3F8802042F00072C3F886
:1005A0008020D3F8802022F00072C3F88020D3F896
:1005B000803072B64FF0E023C3F8084DD4E9000450
:1005C000BFF34F8FBFF36F8F234AC2F88410BFF37E
:1005D0004F8F536923F480335361BFF34F8FD2F8A9
:1005E000803043F6E076C3F3C905C3F34E335B01B5
:1005F00003EA060C29464CEA81770139C2F8747285
:10060000F9D2203B13F1200FF2D1BFF34F8FBFF38C
:100610006F8FBFF34F8FBFF36F8F536923F4003396
:1006200053610023C2F85032BFF34F8FBFF36F8F77
:10063000202383F31188854680F308882047F8BD7E
:100640000000020820000208FFFF0108002200202D
:10065000742200200044025800ED00E02DE9F04F24
:1006600093B0A94B2022FF2100900AA89D6800F0BA
:10067000CFFBA64A1378A3B90121A5481170C36026
:10068000202383F31188C3680BB101F013FE00230C
:10069000A04A4FF47A719E4801F0D0FD002383F305
:1006A0001188009B9C4A03B1136000239B49009C66
:1006B00098469B461E469A460B705360012000F0F8
:1006C0007DFB24B1944B1B68002B00F016820020A8
:1006D00000F082FA0390039B002BF2DB012000F074
:1006E0006BFB039B213B162BE8D801A252F823F0A9
:1006F0004D0700087507000809080008BD06000836
:10070000BD060008BD0600089D0800086F0A000825
:1007100089090008EB090008130A0008390A0008D3
:10072000BD0600084B0A0008BD060008BD0A000807
:10073000ED070008BD060008010B00085907000876
:10074000ED070008BD060008EB0900080220FFF7CE
:100750008DFE002840F0FB81009B022105A8B8F126
:10076000000F08BF1C4641F21233ADF8143000F000
:1007700051FAA3E74FF47A7000F02EFA071EEBDB74
:100780000220FFF773FE0028E6D0013F052F00F29C
:10079000E081DFE807F0030A0D101336052304217A
:1007A00005A8059300F036FA17E004215648F9E74A
:1007B00004215B48F6E704215A48F3E74FF01C098F
:1007C000484609F1040900F057FA0421059005A8EC
:1007D00000F020FAB9F12C0FF2D101204FF0000AFD
:1007E00000FA07F747EA0B0B5FFA8BFB00F05CFBA4
:1007F00026B10BF00B030B2B08BF0024FFF73EFEC6
:100800005CE704214848CDE7002EA5D00BF00B0390
:100810000B2BA1D10220FFF729FE074600289BD011
:1008200001203E4E00F026FA4FF000080220307002
:1008300000F0C4FA5FFA88F9484600F02BFA044643
:1008400090B1484608F1010800F034FA0028F1D1CF
:10085000B846044641F21213022105A83E46ADF8FF
:10086000143000F0D7F929E7012325460220337020
:1008700000F0A2FA244B9B68AB4207D9284600F04F
:10088000FBF9013040F068810435F3E70025234B84
:10089000B8463E461D70204B5D60A7E7002E3FF432
:1008A0005BAF0BF00B030B2B7FF456AF02201B4BFF
:1008B000187000F083FA322000F08EF9B0F10009D0
:1008C000FFF64AAF19F003077FF446AF0E4A09EB73
:1008D0000503926893423FF63FAFB9F5807F3FF73B
:1008E0003BAF124BB945019322DD4FF47A7000F013
:1008F00073F90390039A002AFFF62EAF039A01378B
:10090000019B03F8012BEDE7002200207823002053
:1009100060220020950400087C230020742200201F
:1009200004220020082200200C220020782200202F
:10093000C820FFF79BFD074600283FF40DAF1F2D91
:1009400011D8C5F120020AAB25F0030084494A45BD
:10095000184428BF4A46019200F034FA019AFF2158
:100960007F4800F055FA4FEAA903C9F387027C4992
:100970002846019300F054FA064600283FF46AAF77
:10098000019B05EB830531E70220FFF76FFD00288F
:100990003FF4E2AE00F0AAF900283FF4DDAE0027F4
:1009A000B946704B9B68BB4218D91F2F11D80A9BC0
:1009B00001330ED027F0030312AA134453F8203C4E
:1009C00005934846042205A9043700F019FB814627
:1009D000E7E7384600F050F90590F2E7CDF81490BB
:1009E000042105A800F016F900E70023642104A8FB
:1009F000049300F005F900287FF4AEAE0220FFF763
:100A000035FD00283FF4A8AE049800F065F9059084
:100A1000E6E70023642104A8049300F0F1F800281D
:100A20007FF49AAE0220FFF721FD00283FF494AE38
:100A3000049800F053F9EAE70220FFF717FD0028B9
:100A40003FF48AAE00F062F9E1E70220FFF70EFD05
:100A500000283FF481AE05A9142000F05DF9074697
:100A60000421049004A800F0D5F83946B9E73220F3
:100A700000F0B2F8071EFFF66FAEBB077FF46CAE56
:100A8000384A07EB0A03926893423FF665AE0220AC
:100A9000FFF7ECFC00283FF45FAE27F00307574454
:100AA000BA453FF4A3AE50460AF1040A00F0E4F858
:100AB0000421059005A800F0ADF8F1E74FF47A7035
:100AC000FFF7D4FC00283FF447AE00F00FF90028F0
:100AD00044D00A9B01330BD008220AA9002000F061
:100AE0009FF900283AD02022FF210AA800F090F9AF
:100AF000FFF7C4FC1C4801F05DFB13B0BDE8F08FAC
:100B0000002E3FF429AE0BF00B030B2B7FF424AE29
:100B10000023642105A8059300F072F80746002819
:100B20007FF41AAE0220FFF7A1FC814600283FF4B3
:100B300013AEFFF7A3FC41F2883001F03BFB0598B0
:100B400000F0FCF94E463C4600F0AEF9B6E506462C
:100B50004CE64FF0000AFFE5B8467BE6374679E6FB
:100B60007822002000220020A08601002DE9F84F05
:100B70004FF47A7306460D46002402FB03F7DFF8B4
:100B80005080DFF8509098F900305FFA84FA5A1CD0
:100B900001D0A34210D159F824002A4631460368F7
:100BA000D3F820B03B46D847854205D1074B0120FA
:100BB00083F800A0BDE8F88F0134042CE3D14FF492
:100BC000FA7001F0F7FA0020F4E700BFC823002014
:100BD0001022002058410008002307B502460121D9
:100BE0000DF107008DF80730FFF7C0FF20B19DF829
:100BF000070003B05DF804FB4FF0FF30F9E7000099
:100C00000A46042108B5FFF7B1FF80F00100C0B229
:100C1000404208BD074B0A4630B41978064B53F8DA
:100C20002140014623682046DD69044BAC4630BCB8
:100C3000604700BFC823002058410008A08601007B
:100C400070B50A4E00240A4D01F060FD308028681E
:100C50003388834208D901F055FD2B6804440133E1
:100C6000B4F5003F2B60F2D370BD00BFCA23002053
:100C70008423002001F028BE00F1006000F5003060
:100C80000068704700F10060920000F5003001F04C
:100C90009FBD0000054B1A68054B1B889B1A8342B9
:100CA00002D9104401F02EBD00207047842300209B
:100CB000CA23002038B5074D04462868204401F0B7
:100CC00027FD28B928682044BDE8384001F032BD2E
:100CD00038BD00BF842300200020704700F1FF5082
:100CE00000F58F10D0F8000870470000064991F811
:100CF000243033B100230822086A81F82430FFF73A
:100D0000C1BF0120704700BF88230020014B186835
:100D1000704700BF0010005C244BF0B51A68044611
:100D2000234BC2F30B06120C1F885868BE4293F97E
:100D3000085028D09F89BE4206D101200C2505FB12
:100D40000033586893F9085041F201039A421CD0CD
:100D500041F203039A421AD042F201039A4218D098
:100D600042F203039A4208BF5625621E0B46441EF8
:100D70000A4493420FD214F9016F581C6EB1034616
:100D800000F8016CF5E70020D8E75A25EDE7592572
:100D9000EBE75825E9E7184605E02C2482421C7051
:100DA00001D9981C5D70401AF0BD00BF0010005CB6
:100DB0001422002000207047704700007047000098
:100DC00070470000002310B5934203D0CC5CC4549C
:100DD0000133F9E710BD0000013810B510F9013FEB
:100DE0003BB191F900409C4203D11AB10131013A63
:100DF000F4E71AB191F90020981A10BD1046FCE7EB
:100E000003460246D01A12F9011B0029FAD1704795
:100E100002440346934202D003F8011BFAE77047ED
:100E20002DE9F8431F4D14460746884695F82420BF
:100E300052BBDFF870909CB395F824302BB9202278
:100E4000FF2148462F62FFF7E3FF95F82400414653
:100E5000C0F1080205EB8000A24228BF2246D6B2AC
:100E60009200FFF7AFFF95F82430A41B17441E44EF
:100E70009044E4B2F6B2082E85F82460DBD1FFF787
:100E800035FF0028D7D108E02B6A03EB82038342A9
:100E9000CFD0FFF72BFF0028CBD10020BDE8F8838F
:100EA0000120FBE788230020024B1A78024B1A70BE
:100EB000704700BFC823002010220020F8B5194C4D
:100EC000194800F079FC2146174800F0A1FC24687D
:100ED0001648D4F89020164ED2F80438154D43F039
:100EE0000203114FC2F8043801F064F92046124998
:100EF00000F09CFDD4F890200424D2F8043823F0AC
:100F00000203C2F804384FF4E133336055F8040BA0
:100F1000B84202D0314600F0ADFB013C14F0FF04B2
:100F2000F4D1F8BD70420008C832002040420F00E2
:100F3000B0230020584100087842000838B50B4B18
:100F400004461A780A4B53F822500A4B9D420CD0A3
:100F5000094B002118221846FFF75AFF046001468A
:100F60002846BDE8384000F085BB38BDC8230020C6
:100F700058410008C8320020B023002000B59BB0C3
:100F8000EFF3098168226846FFF71CFFEFF3058342
:100F9000044B9A6BDA6A9A6A9A6A9A6A9A6A9A6AA5
:100FA0009B6AFEE700ED00E000B59BB0EFF309811E
:100FB00068226846FFF706FFEFF30583044B9A6B40
:100FC0009A6A9A6A9A6A9A6A9A6A9B6AFEE700BF64
:100FD00000ED00E000B59BB0EFF3098168226846A0
:100FE000FFF7F0FEEFF30583034B5A6B9A6A9A6A98
:100FF0009A6A9A6A9B6AFEE700ED00E0FEE700004D
:1010000030B50A44084D91420DD011F8013B5840CB
:10101000082340F30004013B2C4013F0FF0384EA53
:101020005000F6D1EFE730BD2083B8ED0268436889
:101030001143016003B1184770470000024A13686A
:1010400043F0C0031360704700440040024A136835
:1010500043F0C0031360704700480040024A136821
:1010600043F0C003136070470078004037B5274C49
:10107000274D204600F0F2FA04F1140000940023FA
:101080004FF40072234900F0B3F94FF40072224983
:1010900004F138000094214B00F02CFA204BC4E9F5
:1010A0001735204C204600F0D9FA04F114000094C2
:1010B00000234FF400721C4900F09AF94FF40072BB
:1010C0001A4904F138000094194B00F013FA194B37
:1010D000C4E91735184C204600F0C0FA04F114009A
:1010E00000234FF400721549009400F081F9144B6D
:1010F0004FF40072134904F13800009400F0FAF93B
:10110000114BC4E9173503B030BD00BFCC2300201C
:1011100000E1F50510250020102B00203D100008EF
:10112000004400403824002010270020102D00200B
:101130004D10000800480040A42400201029002081
:101140005D100008102F002000780040037C30B5AF
:10115000334C002918BF0C46012B18D1314B984253
:101160000FD1314BD3F8E82042F40032C3F8E82025
:10117000D3F8102142F40032C3F81021D3F8103113
:1011800005E02A4B98422FD0294B984238D022684C
:10119000036EC16D03EB52038466B3FBF2F3626826
:1011A000150442BF23F0070503F0070343EA450394
:1011B000CB60A36843F040034B60E36843F0010356
:1011C0008B6042F4967343F001030B604FF0FF33E2
:1011D0000B62510505D512F010221DD0B2F1805FCF
:1011E0001CD080F8643030BD0F4BD3F8E82042F4B7
:1011F0008022C3F8E820D3F8102142F48022BBE714
:10120000094BD3F8E82042F08042C3F8E820D3F835
:10121000102142F08042AFE77F23E2E73F23E0E77F
:1012200068410008CC2300200044025838240020E4
:10123000A42400202DE9F047C66D05463768F469FF
:101240002107346219D014F0080118BF8021E20789
:1012500048BF41F02001A3074FF0200348BF41F0F1
:101260004001600748BF41F4807183F31188281D55
:10127000FFF7DCFE002383F31188E2050AD5202363
:1012800083F311884FF40071281DFFF7CFFE002370
:1012900083F311884FF020094FF0000A14F0200862
:1012A00038D13B0616D54FF0200905F1380A200643
:1012B00010D589F31188504600F050F9002836DA2D
:1012C0000821281DFFF7B2FE27F0800333600023BA
:1012D00083F31188790614D5620612D5202383F38F
:1012E0001188D5E913239A4208D12B6C33B127F02A
:1012F00040071021281DFFF799FE3760002383F374
:101300001188E30618D5AA6E1369ABB15069BDE820
:10131000F047184789F31188736A284695F86410D6
:10132000194000F0B5F98AF31188F469B6E7B062A4
:1013300088F31188F469BAE7BDE8F087F8B5154677
:10134000826804460B46AA4200D28568A1692669D4
:10135000761AB5420BD218462A46FFF733FDA36929
:101360002B44A3612846A3685B1BA360F8BD0CD97E
:10137000AF1B18463246FFF725FD3A46E168304478
:10138000FFF720FDE3683B44EBE718462A46FFF7EA
:1013900019FDE368E5E7000083689342F7B504466A
:1013A000154600D28568D4E90460361AB5420BD2DE
:1013B0002A46FFF707FD63692B4463612846A3684B
:1013C0005B1BA36003B0F0BD0DD93246AF1B01918A
:1013D000FFF7F8FC01993A46E0683144FFF7F2FC68
:1013E000E3683B44E9E72A46FFF7ECFCE368E4E7FF
:1013F00010B50A440024C361029B8460C16002618D
:101400000362C0E90000C0E9051110BD08B5D0E9CC
:101410000532934201D1826882B9826801328260CA
:101420005A1C426119700021D0E904329A4224BF4B
:10143000C368436100F0DAFE002008BD4FF0FF30C2
:10144000FBE7000070B5202304460E4683F31188A5
:10145000A568A5B1A368A269013BA360531CA36161
:1014600015782269934224BFE368A361E3690BB155
:1014700020469847002383F31188284607E0314629
:10148000204600F0A3FE0028E2DA85F3118870BD43
:101490002DE9F74F04460E4617469846D0F81C90A3
:1014A0004FF0200A8AF311884FF0000B154665B102
:1014B0002A4631462046FFF741FF034660B94146C0
:1014C000204600F083FE0028F1D0002383F311882A
:1014D000781B03B0BDE8F08FB9F1000F03D0019085
:1014E0002046C847019B8BF31188ED1A1E448AF3EE
:1014F0001188DCE7C160C361009B82600362C0E9C0
:1015000005111144C0E9000001617047F8B50446B7
:101510000D461646202383F31188A768A7B1A36858
:10152000013BA36063695A1C62611D70D4E90432F7
:101530009A4224BFE3686361E3690BB12046984790
:10154000002080F3118807E03146204600F03EFE7F
:101550000028E2DA87F31188F8BD0000D0E90523FE
:1015600010B59A4201D182687AB9826800210132AD
:1015700082605A1C82611C7803699A4224BFC36846
:10158000836100F033FE204610BD4FF0FF30FBE7D3
:101590002DE9F74F04460E4617469846D0F81C90A2
:1015A0004FF0200A8AF311884FF0000B154665B101
:1015B0002A4631462046FFF7EFFE034660B9414612
:1015C000204600F003FE0028F1D0002383F31188A9
:1015D000781B03B0BDE8F08FB9F1000F03D0019084
:1015E0002046C847019B8BF31188ED1A1E448AF3ED
:1015F0001188DCE7026843681143016003B11847B2
:10160000704700001430FFF743BF00004FF0FF3376
:101610001430FFF73DBF00003830FFF7B9BF0000BE
:101620004FF0FF333830FFF7B3BF00001430FFF73F
:1016300009BF00004FF0FF311430FFF703BF000077
:101640003830FFF763BF00004FF0FF323830FFF74C
:101650005DBF000000207047FFF708BD044B03602A
:1016600000234360C0E9023301230374704700BFC5
:101670008041000810B52023044683F31188FFF74A
:1016800065FD02232374002383F3118810BD00003D
:1016900038B5C36904460D461BB904210844FFF759
:1016A000A9FF294604F11400FFF7B0FE002806DA6E
:1016B000201D4FF48061BDE83840FFF79BBF38BD67
:1016C000026843681143016003B118477047000086
:1016D00013B5406B00F58054D4F8A4381A6811781B
:1016E000042914D1017C022911D11979012312890D
:1016F0008B4013420BD101A94C3002F06DF8D4F8A5
:10170000A4480246019B2179206800F0DFF902B06D
:1017100010BD0000143001F0EFBF00004FF0FF33A8
:10172000143001F0E9BF00004C3002F0C1B80000F5
:101730004FF0FF334C3002F0BBB80000143001F022
:10174000BDBF00004FF0FF31143001F0B7BF000003
:101750004C3002F08DB800004FF0FF324C3002F0F8
:1017600087B800000020704710B500F58054D4F809
:10177000A4381A681178042917D1017C022914D1E0
:101780005979012352898B4013420ED1143001F054
:101790004FFF024648B1D4F8A4484FF44073617932
:1017A0002068BDE8104000F07FB910BD406BFFF726
:1017B000DBBF0000704700007FB5124B01250426F7
:1017C000044603600023057400F184024360294647
:1017D000C0E902330C4B0290143001934FF4407374
:1017E000009601F001FF094B04F69442294604F1EA
:1017F0004C000294CDE900634FF4407301F0C8FF40
:1018000004B070BDA8410008AD170008D11600084B
:101810000A68202383F311880B790B3342F82300E5
:101820004B79133342F823008B7913B10B3342F811
:10183000230000F58053C3F8A41802230374002387
:1018400083F311887047000038B5037F044613B155
:1018500090F85430ABB90125201D0221FFF730FF6D
:1018600004F114006FF00101257700F0CBFC04F1C6
:101870004C0084F854506FF00101BDE8384000F08E
:10188000C1BC38BD10B5012104460430FFF718FF74
:101890000023237784F8543010BD000038B5044687
:1018A0000025143001F0B8FE04F14C00257701F05A
:1018B00087FF201D84F854500121FFF701FF2046C7
:1018C000BDE83840FFF750BF90F8803003F0600368
:1018D000202B06D190F881200023212A03D81F2A2B
:1018E00006D800207047222AFBD1C0E91D3303E04F
:1018F000034A426707228267C3670120704700BF1F
:101900002C22002037B500F58055D5F8A4381A6888
:10191000117804291AD1017C022917D119790123E0
:1019200012898B40134211D100F14C04204602F081
:1019300007F858B101A9204601F04EFFD5F8A44898
:101940000246019B2179206800F0C0F803B030BD49
:1019500001F10B03F0B550F8236085B004460D4645
:10196000FEB1202383F3118804EB8507301D082185
:10197000FFF7A6FEFB6806F14C005B691B681BB114
:10198000019001F037FF019803A901F025FF0246FD
:1019900048B1039B2946204600F098F8002383F3C2
:1019A000118805B0F0BDFB685A691268002AF5D0AD
:1019B0001B8A013B1340F1D104F18002EAE70000E9
:1019C000133138B550F82140ECB1202383F311884E
:1019D00004F58053D3F8A4281368527903EB8203EB
:1019E000DB689B695D6845B104216018FFF768FEFC
:1019F000294604F1140001F025FE2046FFF7B4FE4D
:101A0000002383F3118838BD7047000001F018B936
:101A100001234022002110B5044600F8303BFFF7B7
:101A2000F7F90023C4E9013310BD000010B52023ED
:101A3000044683F311882422416000210C30FFF713
:101A4000E7F9204601F01EF902232370002383F3F7
:101A5000118810BD70B500EB8103054650690E4634
:101A60001446DA6018B110220021FFF7D1F9A069FD
:101A700018B110220021FFF7CBF931462846BDE806
:101A8000704001F011BA000083682022002103F0A9
:101A9000011310B5044683601030FFF7B9F92046F2
:101AA000BDE8104001F08CBAF0B4012500EB8104D0
:101AB00047898D40E4683D43A46945812360002344
:101AC000A2606360F0BC01F0A9BA0000F0B4012587
:101AD00000EB810407898D40E4683D43646905811A
:101AE00023600023A2606360F0BC01F01FBB000014
:101AF00070B5022300250446242203702946C0F84D
:101B000088500C3040F8045CFFF782F9204684F8D6
:101B1000705001F05DF963681B6823B129462046C7
:101B2000BDE87040184770BD037880F88C300523FD
:101B3000037043681B6810B504460BB10421984735
:101B40000023A36010BD000090F88C204368027051
:101B50001B680BB1052118477047000070B590F85D
:101B60007030044613B1002380F8703004F1800215
:101B7000204601F049FA63689B68B3B994F8803055
:101B800013F0600535D00021204601F0F3FC002160
:101B9000204601F0E3FC63681B6813B10621204670
:101BA0009847062384F8703070BD20469847002877
:101BB000E4D0B4F88630A26F9A4288BFA36794F944
:101BC0008030A56F002B4FF0200380F20381002DA1
:101BD00000F0F280092284F8702083F3118800213C
:101BE0002046D4E91D23FFF771FF002383F31188FA
:101BF000DAE794F8812003F07F0343EA022340F2FE
:101C00000232934200F0C58021D8B3F5807F48D0DE
:101C10000DD8012B3FD0022B00F09380002BB2D1C6
:101C200004F1880262670222A267E367C1E7B3F5A5
:101C3000817F00F09B80B3F5407FA4D194F882307F
:101C4000012BA0D1B4F8883043F0020332E0B3F5A1
:101C5000006F4DD017D8B3F5A06F31D0A3F5C06396
:101C6000012B90D86368204694F882205E6894F82F
:101C70008310B4F88430B047002884D04368636789
:101C80000368A3671AE0B3F5106F36D040F602423E
:101C900093427FF478AF5C4B63670223A367002312
:101CA000C3E794F88230012B7FF46DAFB4F888302D
:101CB00023F00203A4F88830C4E91D55E56778E7EE
:101CC000B4F88030B3F5A06F0ED194F8823020467E
:101CD00084F88A3001F0DAF863681B6813B10121D7
:101CE00020469847032323700023C4E91D339CE753
:101CF00004F18B0363670123C3E72378042B10D11E
:101D0000202383F311882046FFF7BEFE85F3118858
:101D10000321636884F88B5021701B680BB1204647
:101D2000984794F88230002BDED084F88B3004235F
:101D3000237063681B68002BD6D002212046984789
:101D4000D2E794F8843020461D0603F00F010AD52F
:101D500001F04CF9012804D002287FF414AF2B4B7A
:101D60009AE72B4B98E701F033F9F3E794F88230C8
:101D7000002B7FF408AF94F8843013F00F01B3D038
:101D80001A06204602D501F00DFCADE701F0FEFB7E
:101D9000AAE794F88230002B7FF4F5AE94F88430F3
:101DA00013F00F01A0D01B06204602D501F0E2FB84
:101DB0009AE701F0D3FB97E7142284F8702083F3AD
:101DC00011882B462A4629462046FFF76DFE85F3EB
:101DD0001188E9E65DB1152284F8702083F311883B
:101DE00000212046D4E91D23FFF75EFEFDE60B220D
:101DF00084F8702083F311882B462A462946204612
:101E0000FFF764FEE3E700BFD8410008D0410008B7
:101E1000D441000838B590F870300446002B3ED00D
:101E2000063BDAB20F2A34D80F2B32D8DFE803F0A2
:101E300037313108223231313131313131313737B7
:101E4000856FB0F886309D4214D2C3681B8AB5FBFB
:101E5000F3F203FB12556DB9202383F311882B464F
:101E60002A462946FFF732FE85F311880A2384F8B3
:101E700070300EE0142384F87030202383F311882F
:101E8000002320461A461946FFF70EFE002383F36F
:101E9000118838BDC36F03B198470023E7E70021DD
:101EA000204601F067FB0021204601F057FB6368E4
:101EB0001B6813B10621204698470623D7E7000088
:101EC00010B590F870300446142B29D017D8062B83
:101ED00005D001D81BB110BD093B022BFBD8002156
:101EE000204601F047FB0021204601F037FB6368E4
:101EF0001B6813B1062120469847062319E0152BCD
:101F0000E9D10B2380F87030202383F3118800235C
:101F10001A461946FFF7DAFD002383F31188DAE742
:101F2000C3689B695B68002BD5D1C36F03B1984729
:101F3000002384F87030CEE7024B0022C3E900335F
:101F40009A60704710310020002382680374054BAB
:101F50001B6899689142FBD25A6803604260106026
:101F6000586070471031002008B5202383F3118892
:101F7000037C032B05D0042B0DD02BB983F31188E0
:101F800008BD436900221A604FF0FF334361FFF739
:101F9000DBFF0023F2E7D0E9003213605A60F3E779
:101FA000002382680374054B1B6899689142FBD833
:101FB0005A6803604260106058607047103100201A
:101FC000054B196908741868026853601A60186133
:101FD00001230374FEF7FAB9103100204B1C30B511
:101FE000044687B00A4D10D02B6901A8094A00F0B9
:101FF00025F92046FFF7E4FF049B13B101A800F088
:1020000059F92B69586907B030BDFFF7D9FFF8E7D8
:1020100010310020691F000838B50C4D044641619D
:102020002B6981689A68914203D8BDE83840FFF770
:102030008BBF1846FFF7B4FF01232C6101462374C0
:102040002046BDE83840FEF7C1B900BF103100207E
:10205000044B1A681B6990689B68984294BF0020E3
:10206000012070471031002010B5084C236820690A
:102070001A6854602260012223611A74FFF790FFEE
:1020800001462069BDE81040FEF7A0B910310020DC
:1020900008B5FFF7DDFF18B1BDE80840FFF7E4BF62
:1020A00008BD0000FFF7E0BFFEE7000010B50C4CD4
:1020B000FFF742FF00F0B4F880220A49204600F002
:1020C0003BF8012344F8180C037400F097FC00233C
:1020D00083F3118862B60448BDE8104000F04CB8A4
:1020E00038310020DC410008EC41000800F01CB948
:1020F000EFF3118020B9EFF30583202282F31188DA
:102100007047000010B530B9EFF30584C4F308043C
:1021100014B180F3118810BDFFF7BAFF84F3118862
:10212000F9E70000034A516853685B1A9842FBD8EC
:10213000704700BF001000E08260022202827047F8
:102140008368A3F17C0243F80C2C026943F83C2C11
:10215000426943F8382C074A43F81C2CC268A3F1A3
:10216000180043F8102C022203F8082C002203F870
:10217000072C7047E503000810B5202383F311886E
:10218000FFF7DEFF00210446FFF746FF002383F33D
:102190001188204610BD0000024B1B6958610F20BA
:1021A000FFF70EBF10310020202383F31188FFF7C3
:1021B000F3BF000008B50146202383F311880820EF
:1021C000FFF70CFF002383F3118808BD49B1064BCC
:1021D00042681B6918605A60136043600420FFF76F
:1021E000FDBE4FF0FF307047103100200368984269
:1021F00006D01A680260506018465961FFF7A4BE05
:102200007047000038B504460D462068844200D16E
:1022100038BD036823605C604561FFF795FEF4E715
:10222000054B4FF0FF3103F11402C3E905220022F0
:10223000C3E90712704700BF1031002070B51C4E73
:1022400005460C46C0E9032301F0B0FB334653F8C2
:10225000142F9A420DD130620A2C2CBF00190A307B
:102260002A60C5E90124C6E90555BDE8704001F0C2
:1022700087BB316A431AE31838BF1C469368A342F0
:1022800002D9081901F08CFB73699A6894420CD842
:102290005A68AC602B606A6015609A685D60121BBA
:1022A0009A604FF0FF33F36170BDA41A1B68ECE72E
:1022B0001031002038B51B4C636998420DD08168FD
:1022C000D0E9003213605A600022C2609A680A4462
:1022D0009A604FF0FF33E36138BD03682246002166
:1022E00042F8143F93425A60C16003D1BDE83840C0
:1022F00001F050BB9A688168256A0A449A6001F02F
:1023000055FB6369411B9A688A42E5D9AB181D1ACF
:10231000206A092D98BF01F10A02BDE83840104437
:1023200001F03EBB103100202DE9F041184C002790
:1023300004F11406656901F039FB236AAA68C11A21
:102340008A4215D81344D5F80C802362D5E90032AF
:1023500013605A606369EF60B34201D101F01AFB68
:1023600087F311882869C047202383F31188E1E7A8
:102370006169B14209D013441B1ABDE8F0410A2B30
:102380002CBFC0180A3001F00BBBBDE8F08100BFC4
:102390001031002000207047FEE700007047000069
:1023A0004FF0FF307047000002290CD0032904D001
:1023B0000129074818BF00207047032A05D805489F
:1023C00000EBC2007047044870470020704700BF10
:1023D000D44200083C2200208842000870B59AB020
:1023E00005460846144601A900F0C2F801A8FEF708
:1023F00007FD431C0022C6B25B001046C5E900344D
:1024000023700323023404F8013C01ABD1B202343F
:102410008E4201D81AB070BD13F8011B013204F8C6
:10242000010C04F8021CF1E708B5202383F311889E
:102430000348FFF767FA002383F3118808BD00BF44
:10244000C832002090F8803003F01F02012A07D123
:1024500090F881200B2A03D10023C0E91D3315E039
:1024600003F06003202B08D1B0F884302BB990F82A
:102470008120212A03D81F2A04D8FFF725BA222A4F
:10248000EBD0FAE7034A426707228267C36701205D
:10249000704700BF3322002007B5052917D8DFE8B1
:1024A00001F0191603191920202383F31188104A0B
:1024B00001210190FFF7CEFA019802210D4AFFF7A2
:1024C000C9FA0D48FFF7EAF9002383F3118803B036
:1024D0005DF804FB202383F311880748FFF7B4F964
:1024E000F2E7202383F311880348FFF7CBF9EBE7EA
:1024F000284200084C420008C832002038B50C4D74
:102500000C4C2A460C4904F10800FFF767FF05F15F
:10251000CA0204F110000949FFF760FF05F5CA720D
:1025200004F118000649BDE83840FFF757BF00BF67
:10253000A04B00203C220020044200081142000869
:102540001C42000870B5044608460D46FEF758FCCC
:10255000C6B22046013403780BB9184670BD324626
:102560002946FEF739FC0028F3D10120F6E70000E8
:102570002DE9F04705460C46FEF742FC2B49C6B252
:102580002846FFF7DFFF08B10A36F6B22849284689
:10259000FFF7D8FF08B11036F6B2632E0BD8DFF87C
:1025A0008C80DFF88C90234FDFF894A02E7846B90A
:1025B0002670BDE8F08729462046BDE8F04701F0C7
:1025C000B5BD252E2ED1072241462846FEF704FC34
:1025D00070B9194B224603F1100153F8040B8B42DA
:1025E00042F8040BF9D11B78073511341370DDE77D
:1025F000082249462846FEF7EFFB98B9A21C0F4B6C
:10260000197802320909C95D02F8041C13F8011B8C
:1026100001F00F015345C95D02F8031CF0D11834D5
:102620000835C3E7013504F8016BBFE7F442000841
:102630001C4200080E430008FC42000800E8F11F9D
:102640000CE8F11FBFF34F8F044B1A695107FCD1FF
:10265000D3F810215207F8D1704700BF0020005274
:1026600008B50D4B1B78ABB9FFF7ECFF0B4BDA68E5
:10267000D10704D50A4A5A6002F188325A60D3F869
:102680000C21D20706D5064AC3F8042102F188328C
:10269000C3F8042108BD00BFFE4D002000200052F9
:1026A0002301674508B5114B1B78F3B9104B1A6924
:1026B000510703D5DA6842F04002DA60D3F81021FE
:1026C000520705D5D3F80C2142F04002C3F80C2183
:1026D000FFF7B8FF064BDA6842F00102DA60D3F880
:1026E0000C2142F00102C3F80C2108BDFE4D002070
:1026F000002000520F289ABF00F58060400400209F
:10270000704700004FF40030704700001020704701
:102710000F2808B50BD8FFF7EDFF00F5003302686E
:10272000013204D104308342F9D1012008BD0020D8
:10273000FCE700000F2870B5054645D8FFF7D8FC28
:10274000224CFFF77FFF0646FFF78AFF4FF0FF336B
:10275000072D6361C4F8143120D82361FFF772FF9D
:102760002B0243F02403E360E36843F08003E3605B
:1027700023695A07FCD42846FFF764FF4FF4003161
:10278000FFF7B8FF00F002F93046FFF78BFFFFF7C5
:10279000B9FC2846BDE87040FFF7BABFC4F8103155
:1027A000FFF750FFA5F108031B0243F02403C4F810
:1027B0000C31D4F80C3143F08003C4F80C31D4F858
:1027C00010315B07FBD4D6E7002070BD002000521B
:1027D0002DE9F84F40EA020305460C461746D80695
:1027E00002D00020BDE8F88F27F01F07DFF8D4B033
:1027F000FFF736FF2744BC4203D10120FFF752FF09
:10280000F0E720222946204601F080FC10B920354F
:102810002034F0E72B4605F120021E68711CE0D140
:1028200004339A42F9D1FFF763FC05F17843234A58
:10283000B3F5801F224B28BF9A4603F1040338BF2B
:102840009046A2F1080228BF9846A3F108033ABFB8
:102850009146DA469946FFF7F5FEC8F80060A5EB09
:10286000040CD9F8002004F11C0142F00202C9F85E
:102870000020221FDAF8006016F00506FAD152F89F
:10288000043F8A424CF80230F4D1BFF34F8FFFF778
:10289000D9FE4FF0FF32C8F80020D9F8002022F00E
:1028A0000202C9F80020FFF72DFC2022214628460D
:1028B00001F02CFC0028AAD030469FE714200052DB
:1028C000102100521020005210B5084C237828B176
:1028D0001BB9FFF7C5FE0123237010BD002BFCD0F0
:1028E0002070BDE81040FFF7DDBE00BFFE4D0020A8
:1028F0000244074BD2B210B5904200D110BD441C27
:1029000000B253F8200041F8040BE0B2F4E700BF36
:10291000504000580E4B30B51C6F240405D41C6F7A
:102920001C671C6F44F400441C670A4C0244236873
:10293000D2B243F480732360074B904200D130BD84
:10294000441C51F8045B00B243F82050E0B2F4E7B5
:1029500000440258004802585040005807B5012270
:1029600001A90020FFF7C4FF019803B05DF804FB44
:1029700013B50446FFF7F2FFA04205D0012201A9DA
:1029800000200194FFF7C6FF02B010BD0144BFF361
:102990004F8F064B884204D3BFF34F8FBFF36F8F27
:1029A0007047C3F85C022030F4E700BF00ED00E0A0
:1029B000034B1A681AB9034AD2F8D0241A60704738
:1029C000004E00200040025808B5FFF7F1FF024B0F
:1029D0001868C0F3806008BD004E0020EFF3098343
:1029E000054968334A6B22F001024A6383F3098880
:1029F000002383F31188704700EF00E0202080F36C
:102A0000118862B60D4B0E4AD96821F4E0610904C1
:102A1000090C0A430B49DA60D3F8FC2042F08072BB
:102A2000C3F8FC20084AC2F8B01F116841F0010148
:102A300011601022DA7783F82200704700ED00E081
:102A40000003FA0555CEACC5001000E0202310B5F8
:102A500083F311880E4B5B6813F4006314D0F1EE1E
:102A6000103AEFF309844FF08073683CE361094B3F
:102A7000DB6B236684F30988FFF7EAFA10B1064B93
:102A8000A36110BD054BFBE783F31188F9E700BF95
:102A900000ED00E000EF00E0F7030008FA03000893
:102AA00070B5BFF34F8FBFF36F8F1A4A0021C2F882
:102AB0005012BFF34F8FBFF36F8F536943F400334E
:102AC0005361BFF34F8FBFF36F8FC2F88410BFF312
:102AD0004F8FD2F8803043F6E074C3F3C900C3F3DC
:102AE0004E335B0103EA0406014646EA817501396B
:102AF000C2F86052F9D2203B13F1200FF2D1BFF39C
:102B00004F8F536943F480335361BFF34F8FBFF34B
:102B10006F8F70BD00ED00E0FEE700000A4B0B4830
:102B20000B4A90420BD30B4BC11EDA1C121A22F037
:102B300003028B4238BF00220021FEF769B953F827
:102B4000041B40F8041BECE7EC440008D44F0020C1
:102B5000D44F0020D44F00207047000070B5D0E95A
:102B6000244300224FF0FF359E6804EB42135101CD
:102B7000D3F80009002805DAD3F8000940F08040B6
:102B8000C3F80009D3F8000B002805DAD3F8000BCE
:102B900040F08040C3F8000B013263189642C3F83E
:102BA0000859C3F8085BE0D24FF00113C4F81C3891
:102BB00070BD000000EB8103D3F80CC02DE9F04399
:102BC000DCF814204E1CD0F89050D2F800E005EB51
:102BD000063605EB4118506870450AD30122D5F836
:102BE000343802FA01F123EA0101C5F83418BDE8CE
:102BF000F083AEEB0003BCF81040A34228BF23468D
:102C0000D8F81849A4B2B3EB840FF0D89468A4F1B3
:102C1000040959F8047F3760A4EB09071F44042F07
:102C2000F7D81C44034494605360D4E7890141F011
:102C30002001016103699B06FCD41220FFF772BAE0
:102C400010B50A4C2046FEF7E3FE094BC4F890305D
:102C5000084BC4F89430084C2046FEF7D9FE074BC9
:102C6000C4F89030064BC4F8943010BD044E0020D8
:102C70000000084044430008A04E0020000004402B
:102C80005043000870B503780546012B5DD1494BD0
:102C9000D0F89040984259D1474B0E216520D3F887
:102CA000D82042F00062C3F8D820D3F8002142F0C7
:102CB0000062C3F80021D3F80021D3F8802042F04D
:102CC0000062C3F88020D3F8802022F00062C3F8AD
:102CD0008020D3F8803000F071FC384BE360384B33
:102CE000C4F800380023D5F89060C4F8003EC02333
:102CF00023604FF40413A3633369002BFCDA012330
:102D00000C203361FFF70EFA3369DB07FCD4122085
:102D1000FFF708FA3369002BFCDA00262846A66084
:102D2000FFF71CFF6B68C4F81068DB68C4F8146810
:102D3000C4F81C68002B3AD1224BA3614FF0FF333B
:102D40006361A36843F00103A36070BD1E4B98420A
:102D5000C8D1194B0E214D20D3F8D82042F0007273
:102D6000C3F8D820D3F8002142F00072C3F8002144
:102D7000D3F80021D3F8802042F00072C3F88020FD
:102D8000D3F8802022F00072C3F88020D3F880208E
:102D9000D3F8D82022F08062C3F8D820D3F80021DD
:102DA00022F08062C3F80021D3F8003193E7074B8B
:102DB000C3E700BF044E0020004402584014004006
:102DC00003002002003C30C0A04E0020083C30C070
:102DD000F8B5D0F89040054600214FF00066204637
:102DE000FFF724FFD5F8941000234FF001128F68ED
:102DF0004FF0FF30C4F83438C4F81C2804EB4312F9
:102E000001339F42C2F80069C2F8006BC2F808099A
:102E1000C2F8080BF2D20B68D5F89020C5F89830AC
:102E2000636210231361166916F01006FBD112209D
:102E3000FFF778F9D4F8003823F4FE63C4F80038BB
:102E4000A36943F4402343F01003A3610923C4F8AA
:102E50001038C4F814380B4BEB604FF0C043C4F883
:102E6000103B094BC4F8003BC4F81069C4F80039A2
:102E7000D5F8983003F1100243F48013C5F8982078
:102E8000A362F8BD2043000840800010D0F89020D5
:102E900090F88A10D2F8003823F4FE6343EA011355
:102EA000C2F80038704700002DE9F84300EB8103B9
:102EB000D0F890500C468046DA680FFA81F9480144
:102EC000166806F00306731E022B05EB41134FF044
:102ED000000194BFB604384EC3F8101B4FF0010137
:102EE00004F1100398BF06F1805601FA03F39169CB
:102EF00098BF06F5004600293AD0578A04F15801D8
:102F0000374349016F50D5F81C180B430021C5F811
:102F10001C382B180127C3F81019A7405369611EEC
:102F20009BB3138A928B9B08012A88BF5343D8F81E
:102F30009820981842EA034301F140022146C8F85C
:102F40009800284605EB82025360FFF76FFE08EBFE
:102F50008900C3681B8A43EA845348341E436401D2
:102F60002E51D5F81C381F43C5F81C78BDE8F883EE
:102F700005EB4917D7F8001B21F40041C7F8001BE7
:102F8000D5F81C1821EA0303C0E704F13F030B4AFC
:102F90002846214605EB83035A60FFF747FE05EB01
:102FA0004910D0F8003923F40043C0F80039D5F8AF
:102FB0001C3823EA0707D7E700800010000400024E
:102FC000D0F894201268C0F89820FFF7C7BD000021
:102FD0005831D0F8903049015B5813F4004004D0C8
:102FE00013F4001F0CBF0220012070474831D0F8B5
:102FF000903049015B5813F4004004D013F4001FD3
:103000000CBF02200120704700EB8101CB68196AD8
:103010000B6813604B6853607047000000EB81033E
:1030200030B5DD68AA691368D36019B9402B84BF35
:10303000402313606B8A1468D0F890201C4402EB84
:103040004110013C09B2B4FBF3F46343033323F0B2
:10305000030343EAC44343F0C043C0F8103B2B686A
:1030600003F00303012B0ED1D2F8083802EB411014
:1030700013F4807FD0F8003B14BF43F0805343F03B
:103080000053C0F8003B02EB4112D2F8003B43F082
:103090000443C2F8003B30BD2DE9F041D0F8906008
:1030A00005460C4606EB4113D3F8087B3A07C3F8F4
:1030B000087B08D5D6F814381B0704D500EB81032C
:1030C000DB685B689847FA071FD5D6F81438DB072A
:1030D0001BD505EB8403D968CCB98B69488A5A683B
:1030E000B2FBF0F600FB16228AB91868DA68904243
:1030F0000DD2121AC3E90024202383F3118821463C
:103100002846FFF78BFF84F31188BDE8F081012387
:1031100003FA04F26B8923EA02036B81CB68002B6C
:10312000F3D021462846BDE8F041184700EB810363
:103130004A0170B5DD68D0F890306C692668E660A9
:1031400056BB1A444FF40020C2F810092A6802F056
:103150000302012A0AB20ED1D3F8080803EB421485
:1031600010F4807FD4F8000914BF40F0805040F084
:103170000050C4F8000903EB4212D2F8000940F0F5
:103180000440C2F800090122D3F8340802FA01F120
:103190000143C3F8341870BD19B9402E84BF4020D4
:1031A000206020681A442E8A8419013CB4FBF6F48E
:1031B00040EAC44040F00050C6E700002DE9F0416D
:1031C000D0F8906004460D4606EB4113D3F8087919
:1031D000C3F80879FB071CD5D6F81038DA0718D5DC
:1031E00000EB8103D3F80CC0DCF81430D3F800E016
:1031F000DA6896451BD2A2EB0E024FF000081A6067
:10320000C3F80480202383F31188FFF78FFF88F32E
:1032100011883B0618D50123D6F83428AB40134259
:1032200012D029462046BDE8F041FFF7C3BC012378
:1032300003FA01F2038923EA02030381DCF8083070
:10324000002BE6D09847E4E7BDE8F0812DE9F84F80
:10325000D0F8905004466E69AB691E4016F4805851
:103260006E6103D0BDE8F84FFEF742BC002E12DAC3
:10327000D5F8003E9F0705D0D5F8003E23F00303A4
:10328000C5F8003ED5F80438204623F00103C5F800
:103290000438FEF759FC300505D52046FFF75EFCE3
:1032A0002046FEF741FCB1040CD5D5F8083813F0E0
:1032B000060FEB6823F470530CBF43F4105343F430
:1032C000A053EB60320704D56368DB680BB120467E
:1032D0009847F30200F1BA80B70226D5D4F890904F
:1032E00000274FF0010A09EB4712D2F8003B03F424
:1032F0004023B3F5802F11D1D2F8003B002B0DDA1B
:1033000062890AFA07F322EA0303638104EB870365
:10331000DB68DB6813B13946204698470137D4F89B
:103320009430FFB29B689F42DDD9F00619D5D4F8DE
:103330009000026AC2F30A1702F00F0302F4F012BF
:10334000B2F5802F00F0CC80B2F5402F09D104EB0C
:103350008303002200F58050DB681B6A974240F02F
:10336000B2803003D5F8185835D5E90303D50021CC
:103370002046FFF791FEAA0303D501212046FFF75F
:103380008BFE6B0303D502212046FFF785FE2F033A
:1033900003D503212046FFF77FFEE80203D5042171
:1033A0002046FFF779FEA90203D505212046FFF745
:1033B00073FE6A0203D506212046FFF76DFE2B023D
:1033C00003D507212046FFF767FEEF0103D508214B
:1033D0002046FFF761FE700340F1A980E90703D59D
:1033E00000212046FFF7EAFEAA0703D50121204667
:1033F000FFF7E4FE6B0703D502212046FFF7DEFE50
:103400002F0703D503212046FFF7D8FEEE0603D58C
:1034100004212046FFF7D2FEA80603D50521204649
:10342000FFF7CCFE690603D506212046FFF7C6FE4E
:103430002A0603D507212046FFF7C0FEEB0576D507
:1034400020460821BDE8F84FFFF7B8BED4F89090A9
:1034500000274FF0010AD4F894305FFA87FB9B688D
:103460009B453FF639AF09EB4B13D3F8002902F423
:103470004022B2F5802F24D1D3F80029002A20DA87
:10348000D3F8002942F09042C3F80029D3F800296C
:10349000002AFBDB5946D4F89000FFF7C7FB2289CE
:1034A0000AFA0BF322EA0303238104EB8B03DB68A4
:1034B0009B6813B159462046984759462046FFF766
:1034C00079FB0137C7E7910701D1D0F80080072ABF
:1034D00002F101029CBF03F8018B4FEA18283DE777
:1034E00004EB830300F58050DA68D2F818C0DCF8EA
:1034F0000820DCE9001CA1EB0C0C00218F4208D154
:10350000DB689B699A683A449A605A683A445A6000
:1035100027E711F0030F01D1D0F800808C4501F1AD
:10352000010184BF02F8018B4FEA1828E6E7BDE8E5
:10353000F88F000008B50348FFF788FEBDE8084093
:10354000FFF784BA044E002008B50348FFF77EFE5B
:10355000BDE80840FFF77ABAA04E0020D0F89030BE
:1035600003EB4111D1F8003B43F40013C1F8003BD9
:1035700070470000D0F8903003EB4111D1F80039CA
:1035800043F40013C1F8003970470000D0F89030C0
:1035900003EB4111D1F8003B23F40013C1F8003BC9
:1035A00070470000D0F8903003EB4111D1F800399A
:1035B00023F40013C1F8003970470000090100F13D
:1035C0006043012203F56143C9B283F8001300F0A0
:1035D0001F039A4043099B0003F1604303F56143D5
:1035E000C3F880211A60704730B50433039C017220
:1035F000002104FB0325C160C0E90653049B03635B
:10360000059BC0E90000C0E90422C0E90842C0E906
:103610000A11436330BD00000022416AC260C0E964
:103620000411C0E90A226FF00101FEF7EBBD0000B2
:10363000D0E90432934201D1C2680AB9181D70471B
:1036400000207047036919600021C2680132C2601E
:10365000C269134482699342036124BF436A0361D0
:10366000FEF7C4BD38B504460D46E3683BB1626958
:103670000020131D1268A3621344E36207E0237A5B
:1036800033B929462046FEF7A1FD0028EDDA38BD02
:103690006FF00100FBE70000C368C269013BC36033
:1036A0004369134482699342436124BF436A43617F
:1036B00000238362036B03B11847704770B5202362
:1036C000044683F31188866A3EB9FFF7CBFF0546AF
:1036D00018B186F31188284670BDA36AE26A13F810
:1036E000015B9342A36202D32046FFF7D5FF00237C
:1036F00083F31188EFE700002DE9F84F04460E46EA
:10370000174698464FF0200989F311880025AA46EC
:10371000D4F828B0BBF1000F09D141462046FFF78D
:10372000A1FF20B18BF311882846BDE8F88FD4E9BA
:103730000A12A7EB050B521A934528BF9346BBF11B
:10374000400F1BD9334601F1400251F8040B91425E
:1037500043F8040BF9D1A36A403640354033A362E5
:10376000D4E90A239A4202D32046FFF795FF8AF351
:103770001188BD42D8D289F31188C9E730465A462C
:10378000FDF720FBA36A5E445D445B44A362E7E768
:1037900010B5029C0433017204FB0321C460C0E92C
:1037A00006130023C0E90A33039B0363049BC0E9AB
:1037B0000000C0E90422C0E90842436310BD0000D4
:1037C000026A6FF00101C260426AC0E9042200226D
:1037D000C0E90A22FEF716BDD0E904239A4201D1BE
:1037E000C26822B9184650F8043B0B6070470020AD
:1037F00070470000C3680021C2690133C360436998
:10380000134482699342436124BF436A4361FEF7D4
:10381000EDBC000038B504460D46E3683BB12369B2
:1038200000201A1DA262E2691344E36207E0237AD2
:1038300033B929462046FEF7C9FC0028EDDA38BD29
:103840006FF00100FBE7000003691960C268013AEC
:10385000C260C269134482699342036124BF436A10
:10386000036100238362036B03B1184770470000B4
:1038700070B520230D460446114683F31188866AED
:103880002EB9FFF7C7FF10B186F3118870BDA36A88
:103890001D70A36AE26A01339342A36204D3E16913
:1038A00020460439FFF7D0FF002080F31188EDE7B0
:1038B0002DE9F84F04460D46904699464FF0200AF0
:1038C0008AF311880026B346A76A4FB949462046B5
:1038D000FFF7A0FF20B187F311883046BDE8F88FCD
:1038E000D4E90A073A1AA8EB0607974228BF1746F9
:1038F000402F1BD905F1400355F8042B9D4240F899
:10390000042BF9D1A36A40364033A362D4E90A23D9
:103910009A4204D3E16920460439FFF795FF8BF3FF
:1039200011884645D9D28AF31188CDE729463A460F
:10393000FDF748FAA36A3D443E443B44A362E5E7F1
:10394000D0E904239A4217D1C3689BB1836A8BB133
:10395000043B9B1A0ED01360C368013BC360C3696C
:103960001A4483699A42026124BF436A03610023B7
:1039700083620123184670470023FBE700F0DAB8A2
:10398000034B002258631A610222DA60704700BFBD
:10399000000C0040014B0022DA607047000C004030
:1039A000014B5863704700BF000C0040014B586A40
:1039B000704700BF000C00404B6843608B68836019
:1039C000CB68C3600B6943614B6903628B694362D7
:1039D0000B6803607047000008B53C4B40F2FF7174
:1039E0003B48D3F888200A43C3F88820D3F88820BE
:1039F00022F4FF6222F00702C3F88820D3F888205F
:103A0000D3F8E0200A43C3F8E020D3F808210A43A2
:103A1000C3F808212F4AD3F808311146FFF7CCFF2D
:103A200000F5806002F11C01FFF7C6FF00F5806021
:103A300002F13801FFF7C0FF00F5806002F1540188
:103A4000FFF7BAFF00F5806002F17001FFF7B4FFE5
:103A500000F5806002F18C01FFF7AEFF00F5806099
:103A600002F1A801FFF7A8FF00F5806002F1C40190
:103A7000FFF7A2FF00F5806002F1E001FFF79CFF75
:103A800000F5806002F1FC01FFF796FF02F58C71F2
:103A900000F58060FFF790FF00F000F90E4BD3F8BF
:103AA000902242F00102C3F89022D3F8942242F00F
:103AB0000102C3F894220522C3F898204FF0605207
:103AC000C3F89C20054AC3F8A02008BD0044025852
:103AD000000002585C43000800ED00E01F000803EE
:103AE00008B500F0F3FAFEF7E1FA0F4BD3F8DC204B
:103AF00042F04002C3F8DC20D3F8042122F0400257
:103B0000C3F80421D3F80431084B1A6842F00802C4
:103B10001A601A6842F004021A60FEF749FFBDE815
:103B20000840FEF7EBBC00BF0044025800180248F2
:103B300070470000114BD3F8E82042F00802C3F8A8
:103B4000E820D3F8102142F00802C3F810210C4AF3
:103B5000D3F81031D36B43F00803D363C722094B6A
:103B60009A624FF0FF32DA6200229A615A63DA6099
:103B70005A6001225A611A60704700BF004402581F
:103B80000010005C000C0040094A08B51169D368B8
:103B90000B40D9B29B076FEA0101116107D52023C1
:103BA00083F31188FEF7A2FA002383F3118808BD7E
:103BB000000C0040384B4FF0FF31D3F88020C3F8A1
:103BC0008010D3F880200022C3F88020D3F8800032
:103BD000D3F88400C3F88410D3F88400C3F8842099
:103BE000D3F88400D86F40F0FF4040F4FF0040F469
:103BF0003F5040F03F00D867D86F20F0FF4020F4DE
:103C0000FF0020F43F5020F03F00D867D86FD3F872
:103C100088006FEA40506FEA5050C3F88800D3F82C
:103C20008800C0F30A00C3F88800D3F88800D3F8EE
:103C30009000C3F89010D3F89000C3F89020D3F808
:103C40009000D3F89400C3F89410D3F89400C3F80C
:103C50009420D3F89400D3F89800C3F89810D3F8C0
:103C60009800C3F89820D3F89800D3F88C00C3F8D4
:103C70008C10D3F88C00C3F88C20D3F88C00D3F8C8
:103C80009C00C3F89C10D3F89C10C3F89C20D3F878
:103C90009C3000F0E7B900BF00440258614B01229C
:103CA000C3F80821604BD3F8F42042F00202C3F8B5
:103CB000F420D3F81C2142F00202C3F81C21022296
:103CC000D3F81C31594BDA605A689104FCD5584A34
:103CD0001A6001229A60574ADA6000221A614FF492
:103CE00040429A61514B9A699204FCD51A6842F499
:103CF00080721A604C4B1A6F12F4407F04D04FF45C
:103D000080321A6700221A671A6842F001021A60AC
:103D1000454B1A685007FCD500221A611A6912F047
:103D20003802FBD1012119604FF0804159605A6778
:103D3000414ADA62414A1A611A6842F480321A60D2
:103D4000394B1A689103FCD51A6842F480521A6004
:103D50001A689204FCD53A4A3A499A6200225A6398
:103D600019633949DA6399635A64384A1A64384ADC
:103D7000DA621A6842F0A8521A602B4B1A6802F0F5
:103D80002852B2F1285FF9D148229A614FF4886233
:103D9000DA6140221A622F4ADA644FF080521A65C3
:103DA0002D4A5A652D4A9A6532232D4A13601368AD
:103DB00003F00F03022BFAD11B4B1A6942F00302E6
:103DC0001A611A6902F03802182AFAD1D3F8DC20F5
:103DD00042F00052C3F8DC20D3F8042142F0005234
:103DE000C3F80421D3F80421D3F8DC2042F0804248
:103DF000C3F8DC20D3F8042142F08042C3F8042148
:103E0000D3F80421D3F8DC2042F00042C3F8DC20D0
:103E1000D3F8042142F00042C3F80421D3F804315E
:103E2000704700BF0080005100440258004802580B
:103E300000C000F0020000010000FF0100889008AF
:103E400032206000630209011D02040047040508D6
:103E5000FD0BFF01200000200010E0000001010028
:103E6000002000524FF0B04208B5D2F8883003F07D
:103E70000103C2F8883023B1044A13680BB15068BB
:103E80009847BDE80840FEF7E1BD00BF544F002051
:103E90004FF0B04208B5D2F8883003F00203C2F800
:103EA000883023B1044A93680BB1D0689847BDE8C5
:103EB0000840FEF7CBBD00BF544F00204FF0B0428A
:103EC00008B5D2F8883003F00403C2F8883023B173
:103ED000044A13690BB150699847BDE80840FEF7E2
:103EE000B5BD00BF544F00204FF0B04208B5D2F826
:103EF000883003F00803C2F8883023B1044A93697C
:103F00000BB1D0699847BDE80840FEF79FBD00BFE0
:103F1000544F00204FF0B04208B5D2F8883003F07B
:103F20001003C2F8883023B1044A136A0BB1506AF7
:103F30009847BDE80840FEF789BD00BF544F0020F8
:103F40004FF0B04310B5D3F8884004F47872C3F84A
:103F50008820A30604D5124A936A0BB1D06A984709
:103F6000600604D50E4A136B0BB1506B98472106BF
:103F700004D50B4A936B0BB1D06B9847E20504D57F
:103F8000074A136C0BB1506C9847A30504D5044A3B
:103F9000936C0BB1D06C9847BDE81040FEF756BD4E
:103FA000544F00204FF0B04310B5D3F8884004F4CC
:103FB0007C42C3F88820620504D5164A136D0BB104
:103FC000506D9847230504D5124A936D0BB1D06DFF
:103FD0009847E00404D50F4A136E0BB1506E984712
:103FE000A10404D50B4A936E0BB1D06E98476204BE
:103FF00004D5084A136F0BB1506F9847230404D5BA
:10400000044A936F0BB1D06F9847BDE81040FEF79C
:104010001DBD00BF544F002008B50348FDF70AF945
:10402000BDE80840FEF712BDCC23002008B50348C8
:10403000FDF700F9BDE80840FEF708BD3824002070
:1040400008B50348FDF7F6F8BDE80840FEF7FEBCEA
:10405000A424002008B5FFF797FDBDE80840FEF74F
:10406000F5BC0000062108B50846FFF7A7FA0621AF
:104070000720FFF7A3FA06210820FFF79FFA062181
:104080000920FFF79BFA06210A20FFF797FA06217D
:104090001720FFF793FA06212820FFF78FFA09214E
:1040A0007A20FFF78BFA07213220FFF787FA0C21DD
:1040B0002620FFF783FA0C212720FFF77FFA0C2137
:1040C0005220BDE80840FFF779BA000008B5FFF7B5
:1040D00071FD00F00DF8FDF7BFFAFDF797FCFDF755
:1040E00069FBFFF725FDBDE80840FFF747BC00006E
:1040F0000023054A19460133102BC2E9001102F1D1
:104100000802F8D1704700BF544F002010B50139A4
:104110000244904201D1002005E0037811F8014FDC
:10412000A34201D0181B10BD0130F2E7034611F87D
:10413000012B03F8012B002AF9D1704753544D335A
:104140003248373F3F3F0053544D333248373433C2
:104150002F37353300000000C8320020CC23002068
:1041600038240020A4240020009600000000000055
:10417000000000000000000000000000000000003F
:1041800000000000211600080D160008491600085E
:1041900035160008411600082D16000819160008EB
:1041A0000516000855160008000000003117000829
:1041B0001D17000859170008451700085117000877
:1041C0003D17000829170008151700086517000893
:1041D0000000000001000000000000006D61696E39
:1041E0000000000069646C6500000000E441000804
:1041F00050310020C832002001000000A920000832
:10420000000000004865782F50726F6669434E4386
:104210000025424F415244252D424C002553455222
:1042200049414C2500000000020000000000000091
:1042300051190008C119000840004000704B0020CF
:10424000804B00200200000000000000030000007E
:1042500000000000091A0008000000001000000023
:10426000904B002000000000010000000000000052
:10427000044E00200101020099240008A92300082F
:10428000452400082924000843000000904200084B
:1042900009024300020100C03209040000010202C9
:1042A000010005240010010524010001042402027C
:1042B0000524060001070582030800FF0904010028
:1042C000020A000000070501024000000705810204
:1042D0004000000012000000DC4200081201100142
:1042E00002000040AE2D1610000201020301000082
:1042F0000403090425424F41524425004375626579
:104300004F72616E67652D626473686F740030313F
:10431000323334353637383941424344454600005C
:10432000000000005D1B0008151E0008C11E0008EB
:10433000400040003C4F00203C4F002001000000A6
:104340004C4F0020800000004001000008000000E9
:104350000001000000040000080000000000812AA5
:1043600000000000AAAAAAAA00000024FFFE000084
:104370000000000000A00A00000100000000000092
:10438000AAAAAAAA00000000FFFF00000000000087
:10439000000000001400005400000000AAAAAAAA0D
:1043A00014000054FFFF00000000000000000000A7
:1043B00000681A0000000000AAAA8AAA005415008A
:1043C000FFFF00000000700777000000408102003E
:1043D00000000000AAAAAAAA00410100F7FF0000FD
:1043E0000000007007000000000000000000000056
:1043F000AAAAAAAA00000000FFFF00000000000017
:10440000000000000000000000000000AAAAAAAA04
:1044100000000000FFFF000000000000000000009E
:104420000000000000000000AAAAAAAA00000000E4
:10443000FFFF00000000000000000000000000007E
:1044400000000000AAAAAAAA00000000FFFF0000C6
:10445000000000000000000000000000000000005C
:10446000AAAAAAAA00000000FFFF000000000000A6
:10447000000000000000000000000000AAAAAAAA94
:1044800000000000FFFF000000000000000000002E
:104490008C0000000000000000001E000000000072
:1044A000FF000000000000003C4100083F00000049
:1044B00050040000474100083F0000000096000043
:1044C0000000080096000000000800000400000042
:1044D000F0420008000000000000000000000000A2
:0C44E000000000000000000000000000D0
:00000001FF
